:040000000202923234
:01000B0032C2
:0100130032BA
:01001B0032B2
:0300230002036372
:100040000D0A0A0A0A0A0A0A0A0A0A0A0A0A0A0A0D
:100050000A0A0A0A0A0A0A0A0A0A41746D656C2029
:100060004154383943383235322053504920507288
:100070006F6772616D6D65722056312E300A0D5FAB
:100080005F5F5F5F5F5F5F5F5F5F5F5F5F5F5F5F80
:100090005F5F5F5F5F5F5F5F5F5F5F5F5F5F5F5F70
:1000A0005F5F0A0D5772697474656E206279205023
:1000B000657465722041766572696C6C2020203110
:1000C0002D372D313939390A0A0A0D50726573738B
:1000D0003A0D0A202020202020206520546F206522
:1000E0007261736520626F746820384B20636F649F
:1000F00065202620324B2064617461206D656D6F30
:1001000072790D0A202020202020206320546F20A7
:10011000646F776E6C6F6164204845582066696C27
:100120006520746F20636F6465206D656D6F7279F3
:100130000D0A202020202020206420546F20646F8E
:10014000776E6C6F6164204845582066696C652045
:10015000746F2064617461206D656D6F72790D0A32
:10016000202020202020206C20546F20777269747A
:1001700065206C6F636B20626974730D0A000A0D51
:100180004845582066696C65207265636F7264200B
:100190006572726F722C2070726573732072657352
:1001A000657420746F20726573746172742070724C
:1001B0006F6772616D6D6572000A0D5265636F72D3
:1001C00064206661696C656420746F20766572696D
:1001D00066792C2070726573732072657365742064
:1001E000746F20726573746172742070726F6772BD
:1001F000616D6D6572000A0D50726F6772616D6D91
:10020000696E672066696E697368656420707265DF
:10021000737320616E79206B657920746F2072652D
:100220007475726E20746F206D61696E206D656EDD
:1002300075000A0D5461726765742070726F636592
:1002400073736F722072657365742072656C65617B
:100250007365640A0D507265737320616E79206B4B
:10026000657920746F2072657475726E20746F20CA
:100270006D61696E206D656E75000A0D53656E6463
:1002800020746578742066696C65206E6F770D0A3E
:100290000A0075815F120371D29990004012039099
:1002A0001203AF1203A7B46503120501B46303126E
:1002B00002C0B464031202C6B46CDF1202CC80DA4E
:1002C000D2201202E622C2201202E622120518747F
:1002D000AC1204D374071204D374551204D3740AF5
:1002E00012052FC2942290027A120390C2ACD299C6
:1002F000C2D51203AF1203A7B43AF71203ED5003AD
:10030000020339B4002B74131203A720D50512057C
:1003100018D2D512043C120484402B74561203A741
:10032000740D1203A7740A1203A774111203A78095
:10033000C112052CC2D502035390017E12039074A2
:10034000111203A780FE9001B912039074111203D9
:10035000A780FE9001F61203901203AF2098FA12C4
:1003600003AF22C2D5C299309806E599D2D5C2987A
:100370003275870075A800759840758921758DFDC7
:10038000758840D29CD2AFD296D295C297C29422A1
:10039000C0E0C082C083E49360061203A7A380F686
:1003A000D083D082D0E0223099FDC299F5992220E5
:1003B00098033098FDE599C2982271AF71A7120396
:1003C000D2400EC4F5F071AF71A71203D2400245BE
:1003D000F022FEC3943A5007EEC394300203ECEED1
:1003E0009447B34007EE94414002240A227D0071F5
:1003F000BA4047F533C39411504071BA403CF532CE
:1004000071BA4036F53171BA4030F530B400117828
:1004100034AF3371BA4023F62DFD08DFF602042510
:10042000E530B4011571BA40112D2533253125323F
:1004300025307006E530C302043BD322AA31AB322B
:10044000EB541F23232330200544020204504406AA
:10045000FE7834AF33EE1204D3EA1204D3E612046A
:10046000D3740312052FEA2401FA5014EB2401FB84
:10047000541F232323302005440202047F4406FE38
:1004800008DFD222AA31AB32EB541F2323233020C2
:100490000544010204984405FE7834AF33EE12049B
:1004A000D3EA1204D31204EB86F0B5F0030204B4CD
:1004B000D30204D2EA2401FA5014EB2401FB541FA6
:1004C00023232330200544010204CD4405FE08DF28
:1004D000CCC322C0F075F0083392950000D297008B
:1004E000000000C297D5F0F0D0F022C0F075F008FF
:1004F000D297A296330000C2970000D5F0F2D0F058
:100500002212051874AC91D3740491D3745591D30D
:10051000740A12052FC29422D294740112052F740A
:10052000AC91D3745391D3745591D322C29422C009
:10053000E0C0F075F000D5F0FDD5F0FDD5E0F7D0C6
:10054000F0D0E022C0E0C0F0F5F074FAB12FB12F86
:0C055000B12FB12FD5F0F3D0F0D0E02295
:00000001FF
